S00E0000427574746F6E2E737265639A
S11300000C942B000C9453000C9453000C94530048
S11300100C94D5000C9453000C9453000C9453008E
S11300200C9453000C9453000C9453000C94530000
S11300300C9453000C9453000C9453000C945300F0
S11300400C9453000C9453000C9453000C945300E0
S11300500C945300DF0011241FBECFE5D8E0DEBFAF
S1130060CDBF10E0A0E6B0E0EEEFF1E002C00590F5
S11300700D92A236B107D9F720E0A2E6B0E001C0A4
S11300801D92A636B207E1F710E0C6E5D0E004C041
S11300902297FE010E94F900C435D107C9F70E94D6
S11300A09B000C94FD000C94000080FF02C0A89AF1
S11300B001C0A898A09A81FF02C0A99A01C0A9987A
S11300C0A19A82FF02C0AA9A01C0AA98A29A08958E
S11300D0CF92DF92EF92FF920F931F93CF93DF9310
S11300E0D82EC62EC0E0D0E019C08D2D0E94550038
S11300F01F5F1F3FD1F700E010E005C08C2D0E9468
S113010055000F5F1F4F0C171D07C4F3FA9411F02D
S11301101E2DEBCF2196CF3FD10521F0EC2E85E0AB
S1130120F82EF6CFDF91CF911F910F91FF90EF90B2
S1130130DF90CF9008951AEACEEFD3E610936200D1
S1130140C0936300D09364002FEF86E191E12150C6
S113015080409040E1F700C00000C0936200C0936B
S11301606300C09364002FEF86E191E12150804049
S11301709040E1F700C0000066E084E00E9468005F
S113018062E086E00E94680063E082E00E9468000A
S113019061E083E00E94680065E081E00E946800FD
S11301A064E085E00E946800C9CF1F920F920FB6E9
S11301B00F9211240F900FBE0F901F901895A59ABF
S11301C0AD98A59AA49AAC98A49A10926200109241
S11301D0630010926400A29AA19AA09A12BC85E0CE
S11301E085BD14BC13BC80E889BF78940895EE0FD4
S11101F0FF1F0590F491E02D0994F894FFCFC1
S10501FE0100FA
S9030000FC
